:030000000219FDE5
:03000B000200A848
:03002B000201636C
:03005B000202EDB1
:030073000202D3B3
:1000800002030406080C10182030406080040608A3
:100090000C10182030406080A0C000070F1F3F05E3
:1000A000050D050305030302C2AFC0D0C0E0206206
:1000B00017E5256002E473E525F4F58A758B00D217
:1000C00062D0E0D0D0D2AF3285268AC262E526F473
:1000D0006035306803207210758B00D0E0D0D0C23C
:1000E000B1C287C281D2AF32C2B1C287C281206E93
:1000F0000C206609740AD5E0FDE57E4280758B0010
:10010000D0E0D0D0D2AF32758A00C28DD26201FD6C
:1001100001B7306805206602D2B101B7306805200A
:100120006602D28701B7306805206602D28101B726
:10013000C28230680A2066077408D5E0FDD2B1019A
:10014000B7C28630680A2066077408D5E0FDD287FA
:1001500001B7C28030680A2066077408D5E0FDD276
:100160008101B7C2AFC2AD53E6EFC0D0C0E0D2D379
:10017000D2AFC2CEE52A6007207449152A21C4787F
:1001800000790020742EE580307E01F430E502789D
:10019000FF53DACF207E0343DA20307E0343DA10A8
:1001A000C2D8C271E580307E01F430E50279FFC328
:1001B000E89970CB306103752A18207403752A18EA
:1001C000885FD27020740DE52B6004152B21D44379
:1001D000DA01C2D82070024136A85F206102C270E5
:1001E000207431C3E894F0400374F0F8E8C4540F6D
:1001F00028F87984B703024114C313C3138721205D
:100200000802C313200A06C3C898F8411428F850FE
:100210000374FFF8C3E895685003E568F88822E5A1
:100220002D54066011E533C313C31324062522F5AC
:100230002250037522FF852224A824C3E524956457
:100240004002A8648825E5697002417AC3E8AA697A
:100250009A5003E8FAE4F9EAC333FBE56BF45B294F
:10026000400D256AF8E56A6002156A400B417A0A7A
:10027000C3E56A9A5002056A78FF8826C26EC3E514
:100280002694F84002D26EC3E52594404002D26421
:1002900020CF0AD0E0D0D043E610D2AD32C2CF0595
:1002A0003A7801E52A6005307402152AC3E55F94A7
:1002B00001400575620041C9756300756C00E56217
:1002C0002401F56250037562FFD0E0D0D043E61000
:1002D000D2AD32C2AFC0D053E67FC2607591008507
:1002E0005694855795759104D0D0D2AF32C2AF5392
:1002F000E6EFC2ADC0D0C0E0C0F0D2D3D2AFA8FB11
:10030000A9FCC2D8307102615453DACF207E034376
:10031000DA10307E0343DA20D271E580307E01F4BA
:1003200020E502612B88278928A17B53DACF207E24
:100330000343DA20307E0343DA10C2D8C27130742E
:1003400002A1677800E580307E01F430E502A16704
:10035000885FA14F53DACF207E0343DA20307E033B
:1003600043DA10C271206102812D53DACF207E035F
:1003700043DA10307E0343DA20C2D8D271885A891A
:100380005BC3E89558F8E99559F97B007E087A0037
:10039000C3E8948CE994005005755E00811F8821A4
:1003A00078A2E6A8216055C3E894C8E994005008F3
:1003B000E4D2E4FB7A0A61FAC3E89468E994015054
:1003C00008E4D2E3FB7A0F61FAC3E894D0E994021F
:1003D0005008E4D2E2FB7A1E61FAC3E894A0E994E3
:1003E000055008E4D2E1FB7A3C61FAC3E89498E94D
:1003F00094085008E4D2E0FB7A787E00C3E8955C6C
:10040000FCE9955DFD30E70AECF42401FCEDF434E1
:1004100000FD755E00C3EC9AED9E5003755E018889
:100420005C895D855A58855B597802A14FC3E89570
:1004300027F8E99528F9307C02A133307B02A133FB
:10044000307A02A12C2075028150E9FDE8FC816F11
:10045000E9C313F9E813F8307902A12CE9C313F9C1
:10046000E813F8307802A12CE9C313FDE813FC204F
:0E0470006126C3EC941CED940240028186EDDF
:10047E007018C3EC94C850120529C3E529940A508C
:10048E0002A167755F00D270A167E5296002152988
:10049E007888E6F97400207F087896B90302789E72
:1004AE00E624FAFEE43400FFC3EC9EFCED9FFD92C1
:1004BE0008B90310A2085007207609D27681D230EF
:1004CE007602C276A2085016B9030DECF42401FC94
:1004DE00EDF43400FD0204EC78007900A133B90389
:1004EE0015EC33FCED33FDC3EC940AFCED9400FDEA
:1004FE0050047C007D00C3EC94FFED940040067820
:10050E00FF7900A133EC8575F0A4C5F0A2F733F89E
:10051E007900400302054F78FF790002054FE9C3C9
:10052E0013F9E813F8307C0EE9600278FFC3E81384
:10053E0038F8E43400F9C3E894FFE99400400278F7
:10054E00FF885FD270206102A167741FF4552F4B94
:10055E00F52FC274EB7002D274752A1830740375BD
:10056E002A0A306102A17B20740353DAFE20740341
:10057E00752B06D0F0D0E0D0D0D2AD43E610327954
:10058E00010205AB79030205AB790A0205AB791EB0
:10059E000205AB79640205AB79C80205AB7817E4A6
:1005AE00D5E0FDD8FAD9F6227A147B780205D27AF4
:1005BE00107B8C0205D27A0D7BB40205D27A0B7BAE
:1005CE00C80205D27902B27DE4C286D5E0FDD2879B
:1005DE00D5E0FDC287D5E0FDD286D5E0FDD2B1E5EE
:1005EE0076D5E0FDC2B17496D5E0FDD9D9EAF8D53D
:1005FE00E0FDD8FBDBCEC28622C37C007D0075F009
:10060E000005F0EA33FAEB33FB50F6EB13FBEA137B
:10061E00FAC3E9FFE8FEE89AF8E99BF95004EFF90E
:10062E00EEF8B3EC33FCED33FDD5F0DFEDF9ECF87D
:10063E0022E889F08A20D2D4F8A9F07B0030F70B9B
:10064E007BFFF42401F8E9F43400F9E88520F0A4E6
:10065E00ADF0F8E98520F0A4AFF0FEED2EF97400B0
:10066E003FFA7C04C3EA13FAE913F9E813F8DCF451
:10067E008BF030F70AE8F42401F8E9F43400F9E8D5
:10068E0089F0C2D4F8A9F02222C3E54113F9E5405E
:10069E0013F8C3E54598F8E54699F9500CC3E8946C
:1006AE0080E994FF40160206CEC3E8947FE99400D9
:1006BE0050030206CE787F79000206CE788079FF4D
:1006CE00884A894B22E54A2547F8E54B3548F98596
:1006DE004B20E4300701F43549FA30E709C3EA94B8
:1006EE00F0401502070CC3EA940F500302070C7872
:1006FE00FF79FF7A0F02070C780079007AF0C3E5D4
:10070E00249564500AC374019524500B02072AE500
:10071E004B20E70E02072AE54B30E706884789484B
:10072E008A492278A4E6FAC3E54A33F8E54B33F951
:10073E00D13FE930E70BC3E89480E994FF4013E121
:10074E0064C3E8947FE994005002E164787F7900F5
:10075E00E164788079FFE820E715C3E52398F84037
:10076E0009C3E89401400302078B780102078BE866
:10077E00F424012523F8400302078B78FF884C22CE
:10078E0078A5E6FAA848A949D13FE930E70CC3E8B5
:10079E009401E994FF40160207BFC3E894FFE99461
:1007AE000050030207BF78FF79000207BF78017976
:1007BE00FFE920E715C3E54C98F84009C3E894011A
:1007CE0040030207E678010207E6E8F42401254C0F
:1007DE00F840030207E678FF88242278FFC26420DF
:1007EE00693D206A12D264C3E541940A4009C3E50B
:1007FE002594405002C26479A1E76023E541601F51
:10080E0074FF8541F0848539F0306A0375F005A4D4
:10081E00F8C5F0600278FFC3E895675002A86788B4
:10082E006622C3E5409440E5419401E56650031409
:10083E000141046002F566220208492275E8902201
:10084E007883E6FFE5E820ECF7A8BDA9BE0573C3E3
:10085E00E57394084052757300E9FA79A0E7604495
:0E086E00EA7007E574601B020884C3E8957405
:10087C006010E5745006600C140208900460F902D4
:10088C000890E574F574C394A8401B7564C0C394B8
:10089C00054013756480C39405400B756440C39484
:1008AC0005400375640075BB0622E564F46002051F
:1008BC0064E573B4070375BB1E22743279A687F006
:1008CC00A4C5F0A2F733F8C3E895644002A8648885
:1008DC00228824882588268867227540007541F077
:1008EC0022C2AF75C820A8CCA9CDAA3A30CF010A34
:1008FC0075C824D2AFAB3BAC3C883B893CC3E89B6E
:10090C00F8E99C206908F93067024102215FAD3D8E
:10091C008A3DF9EA9DFA600478FF79FFAE3EAF3F5D
:10092C008B3E8C3FC3EC9FFCC3E99CF542A83BA9D2
:10093C003CC3E89EF8E99FF9C3E54113FBE540137E
:10094C00FAE82AF540E93BF54150067540FF754140
:10095C00FF21A9AA40AB41AC40AD417E047F02C34C
:10096C00EB940440021E1FC3EB940840021E1FC3ED
:10097C00ED13FDEC13FCDEF7C3EA9CFAEB9DFBEFE9
:10098C006009C3E913F9E813F8DFF7EA28FAEB3941
:10099C00FB8A408B4150067BFF8B408B41C3EB9411
:1009AC00025002D2673069047F0321D47892E6FFAB
:1009BC00C3E537948240110FC3E53794A040010F73
:1009CC00C3EF940640027F057E05E541C4540FF940
:1009DC00E541C454F0F8E540C4540F28F8C3E89E30
:1009EC00FAE99400FB4009C3EA9402EB940050042A
:1009FC007A02E4FB414EAA40AB41EBC4FEEAC4547C
:100A0C000F4EFCC3EA9CFAEB9400FBC3E813C31330
:100A1C00F8EA28FAEB3400FB8A408B41C3EB9402D2
:100A2C004002C2677805EBC4FE7B00EAC4540F4E4B
:100A3C00FAC3EA98FA4005C3940250027A027892FB
:100A4C00E6FF306002414E855256855357D26043C3
:100A5C00E680C3E49AF8E49BF930670241E8E8FACF
:100A6C00E9FBD3E913FDE813FC88528953C3EF94D7
:100A7C00036038EF20E00DE82CF8E93DF9ECFAEDD5
:100A8C00FB020AA3E828F8E939F9C3E82402F8E9DB
:100A9C003400F97AFE7BFFC3EF9403400E8A548B2B
:100AAC0055884E894F8C508D51611C885489558ABC
:100ABC004E8B4F8C508D51306920C3E533940340DD
:100ACC0019E542A2E713F8E555F4240138400B2050
:100ADC00E7087554FFF42401F555611CE8FAD3E8D6
:100AEC0013FC8852C3EF94036020EF20E007E82C3E
:100AFC00F8ECFA6108E8282402F87AFEC3EF9403B4
:100B0C0040088A54884E8C50611C88548A4E8C50F4
:100B1C00E56BC3335002646BF56B30600261267574
:100B2C003402D26043E680E52D54066026A840A925
:100B3C0041C3E913F9E813F8C2AF53E67F7591008E
:100B4C00C3E498F594E499F595759104D26043E665
:100B5C0080D2AF22D265754400752000306B0375CE
:100B6C002040020B7FD265754400752040306B032A
:100B7C00752000D2AF7801206722E52D5406600263
:100B8C00C265C3E54194054013780294054008788A
:100B9C0003940540027806306902780A206019E552
:100BAC0044601530690AC3E53394034003D5340619
:100BBC00D2AFD26C8150712ED2AF0000C2AF206781
:100BCC0026E541C3FB940F40027B0FEB24053073E9
:100BDC000123306A02742820620123F930690279FA
:100BEC0082E58BC39940B50544E59B5440B5200282
:100BFC00813A30690A08C3E8940A40010861A820C8
:100C0C006502617FC26553E67F7591003067107590
:100C1C0094007595FE759104D26043E680617FAEB9
:100C2C0040AF41C3E49EF594E49FF5958121C3E563
:100C3C003394025002617F306502617FD802814E8D
:100C4C0061A8C26C53E67F759100855494855595C7
:100C5C00759104854E56854F57D26043E680D2AFCE
:0E0C6C00E52D54066008206A020533020C8A4A
:100C7A00306C0D206B0A206507158115810215223B
:100C8A002278003064053065027801E53775F0078F
:100C9A00A4F9E5F028F5F0E9A2F013A2F113A2F203
:100CAA0013F537C394785003753778C3E537953809
:100CBA004008D266C2B1C287C28130600281C4854F
:100CCA005056855157D26043E68022207D11C2AF2B
:100CDA00754302C286D282D2AF759F02020EA4C2A7
:100CEA00AF754302C286D280D2AF759F02020EA4AC
:100CFA00307243207D20C2AF754303900141757E57
:100D0A0040C281C280306204D287A118D286D2AF93
:100D1A00759F03020EA4C2AF754303900141757E0D
:100D2A0040C2B1C282306204D287A138D286D2AF21
:100D3A00759F01020EA4207D17C2AF75430390016F
:100D4A001CC281306202D287D2AF759F03020EA401
:100D5A00C2AF75430390011CC2B1306202D287D27E
:100D6A00AF759F01020EA4207D11C2AF754304C264
:100D7A0082D280D2AF759F01020EA4C2AF7543041E
:100D8A00C280D282D2AF759F03020EA43072432072
:100D9A007D20C2AF754305900130757E04C287C2BB
:100DAA0086306204D2B1A1B4D282D2AF759F020258
:100DBA000EA4C2AF754305900152757E01C287C267
:100DCA0086306204D281A1D4D280D2AF759F02024A
:100DDA000EA4207D17C2AF754305900112C2873059
:100DEA006202D2B1D2AF759F02020EA4C2AF75439E
:100DFA0005900126C2873062EBD281D2AF759F027D
:100E0A00020EA4207D11C2AF754306C280D286D2DB
:100E1A00AF759F03020EA4C2AF754306C282D28683
:100E2A00D2AF759F01020EA4307242207D20C2AF5C
:100E3A00754301900152757E01C2B1C282306204CB
:100E4A00D281C150D280D2AF759F01020EA4C2AF27
:100E5A00754301900130757E04C281C280306204FC
:100E6A00D2B1C170D282D2AF759F03C1A4207D16C0
:100E7A00C2AF754301900126C2B1306202D281D25B
:100E8A00AF759F01C1A4C2AF754301900112C2811F
:100E9A00306202D2B1D2AF759F03C26622900110AE
:100EAA00757E00C2B1C287C281C282C286C280C2B6
:100EBA006222788076FF0876FF0876FF0876FF08B8
:100ECA007603087604087609087603087601087618
:100EDA0001788C76010876FF0876FF0876FF087697
:100EEA00FF0876FF0876030876FF0876FF0876FF84
:100EFA000876250876D00876FA0876FA087604087D
:100F0A0076FF08760108760008767A0876FF087672
:100F1A0001087601087600087603227887E6FFC280
:100F2A0072BF0302D2727888E6C394036008C27D56
:100F3A00E630E102D27DC27E7889E630E102D27ED5
:100F4A00C3EF94026008758E01D273020F5D758E2D
:100F5A0000C273227880E6149000809378A4F67811
:100F6A0081E6149000809378A5F67886E6149000BE
:100F7A008D9378A6F6789CE67538FF75390CB4021D
:100F8A00067538A075390AB40306753882753905AD
:100F9A0078A3E61490009A93F569D1A722C2B37890
:100FAA009DE66002D2B3227896E6FA7897E6FB7855
:100FBA0088E6B40305C3EB940EFB307F047A007B0A
:100FCA00FFC3EB9AFCC3948250027C8275750005BC
:100FDA0075EC8575F0A4C3E5F0947D40F222D27FCA
:100FEA00F1B112059C7A007B007C10120592E55F34
:100FFA002AFA74003BFBDCF37C04C3EB13FBEA1311
:10100A00FADCF7FEC27F120FB122E5EF20E6037584
:10101A0020000520903DFFE520146006901FFF1474
:10102A0060009304600375EF1253D9BF7581C04302
:10103A00FF8012058D75EF0243B203E5B324042045
:10104A00E70DF521E5B120E0068521B343B1011290
:10105A000EA775803875A4C775F1FF75D4DF759032
:0D106A00FF75A50075F20075D50075A0FF9B
:1010770075A60075F30075D60075B0E475A71B75E6
:10108700F4FF75E241E4F8F6D8FD756B01120EBC6A
:1010970012156478988676753001C2AF1205A612CC
:1010A70005B612059C1205BD12059C1205C4120552
:1010B7009C12167D1205A61205A61205A1C2AF78CD
:1010C700FA79FA308507D9FBD8F7021C00120F25E9
:1010D700120F5E120FA7120FB178988676120EA71D
:1010E70075885075891275C82475910475D840752F
:1010F700A82275B80275E690759B80759D0075D11D
:101107000E75BC5875BB0675BA1F75E88012058D3C
:10111700D2AF12084653DACF207E0343DA20307E5F
:101127000343DA1043DA01C2D8C2711205A6D261AD
:101137007B037A0CE55E70077A0CDB030210C4129E
:10114700059C2070030210C4C270E55FC39402407F
:10115700E1E52F541F856160F561B560D5DAD5C229
:101167006153DACF207E0343DA20307E0343DA105F
:10117700C2D8C27178A2E67008D274E52F54E0F5A0
:101187002FC2757529001205A1307409C3E529948A
:101197000A4002D27512059278023074027800C3B1
:1011A700E55F9840F0C2AF1205B61205B61205B654
:1011B700D2AF1205A6754D007888E6B4030241A4A4
:1011C700120592788CE6C3940150030212A4E5300D
:1011D700C3940150030212A4207435C3E55F94FF42
:1011E70050030212A4C2AF1205CBD2AF1205A1C39E
:1011F700E55F940150EFC2AF1205B61205971205CD
:10120700B6D2AF1205A1C3E55F94FF40E90217020A
:101217007F05D27F120FB11205A1C2AFC27F120F95
:10122700B1AE5FC3E55F947FD2AF407B12058DC23D
:10123700AF1205CBD2AFDFDA120FE8C3EE94057811
:1012470097F61205A61215A61216857F0AD27F12E7
:101257000FB11205A1C2AFC27F120FB1AE5FC3E5D6
:101267005F947FD2AF50E412058DC2AF1205B6125C
:1012770005971205B6D2AFDFD4120FE8EE24057832
:1012870096F61205A61215A61216B41205A1120F8C
:10129700B1C3E55F94FF500221DF021702C3E55F88
:1012A700954D4003855F4D1205A178017988E7B414
:1012B70003027805C3E55F98400221BFC2AF12055C
:1012C700CB1205CB1205CBD2AF1205A6753000E4C1
:1012D700F531F5320531E531F470390532789AE6A2
:1012E7007819146012783214600D787D14600878CC
:1012F700FA146003753200C3E5329840171532754A
:1013070031B478998676C2AF1205CBD2AF7898867A
:10131700761205A1120597E52A700530740201C4FB
:1013270078012074027806C3E55F9840A77888E6BD
:10133700C3940360031205A1E52A70030210C4C217
:10134700AF120EA7E4F522F523F524F525F526F5CA
:101357006AD2AF7885E6C333F568E4F545F546F517
:1013670047F548F549F573F52CF52DF537757308ED
:1013770075BB1E12058D12084AE5E820ECFBA8BDD7
:10138700A9BEE97001F8887412084E75730875BB19
:101397001E7887E6FE7602120F257887EEF6C2AF33
:1013A7007564FF1208C6852264852265852266D288
:1013B700AF75220175240175250175260185636CBA
:1013C700756D017888E6B40307C27D307602D27D59
:1013D700D268D269753300120E0D120E321208E66A
:1013E7001208ED1208E61208ED1208E6021403C20D
:1013F700AF120F25D2AF75730075BB06120B7112B2
:101407000696120C8B120CD51208ED120B60306D7C
:10141700031206972067031207E9306703120830A3
:10142700120C8B120CFA1208ED120B71306D0312AD
:1014370006D3120C8B120D711208ED120B60306D72
:1014470003120731120C8B120D961208ED120B7155
:10145700306D0312078E120C8B120E0D1208ED124F
:0E146700084A120B60120C8B120E3212084E45
:101475001208ED306932206B2F85676485676585B5
:10148500636C756D0179187A0CC3E53399400CC20C
:1014950069D26A8A357564FF0214ADC3E55F9401AC
:1014A500400302140302152A306A1B206B18E53528
:1014B500147004C26A61F6F535C3E55F9401400313
:1014C50002140302152A753600C3E5627882985026
:1014D50054307404E52A604D7888E6B40317207DFE
:1014E5000520760781FA30760281FA206B07D26BE8
:1014F500856764814278F0306B058567647820C321
:10150500E5419850028103306B1BC26BC27D30767A
:1015150002D27DD26A75351285676481030536E589
:101525005F6002A12D753600C2AF120EA77887E65F
:10153500FE7602120F257887EEF6E4F522F523F5FF
:1015450024F525F526F568C268D2AF12058D120E71
:10155500A7307409C3E5369405400201C441D6900D
:101565001A0D78201215E8E520B45A0CA31215E8D7
:10157500E520B4A503021586120EBC1215A60215A8
:10158500A5901A0378807B0A1215E8A308DBF99069
:101595001A0F788C7B181215E8A308DBF9901A2727
:1015A50022C2AF121627121601901A00740E1215D8
:1015B500EDA374041215EDA374141215ED901A031E
:1015C50078807B0A1215ECA308DBF9901A0F788C4A
:1015D5007B181215ECA308DBF912163A12161890AF
:1015E5001A2722E493F622E6438F01538FFD75EF08
:1015F5000275B7A575B7F1F0538FFE22438F0243ED
:101605008F0175EF0275B7A575B7F1901A0DF053F7
:101615008FFC22901A0D745AB1ED901A0E74A5B173
:10162500ED227A3079D07820901A40B1E8E520F79C
:1016350009A3DAF7227A3079D0901A40E7B1ED099B
:10164500A3DAF922AB77A878BB01027984BB020241
:101655007985BB03027986BB04027992BB050279C1
:1016650087BB060279A3BB0702799CBB0802798870
:10167500BB09027989E8F7227C051205A6DCFB2265
:10168500C2AF1205B61205BD1205C41205CB12056F
:10169500971205B61205BD1205C41205CB120597A2
:1016A5001205B61205BD1205C41205CBD2AF22C272
:1016B500AF1205CB1205C41205BD1205B61205976A
:1016C5001205CB1205C41205BD1205B612059712F7
:1016D50005CB1205C41205BD1205B6D2AF22AE77F1
:1016E500AF78C2AF1205B61205B61205B612059748
:1016F500DEF21205CB120597DFF8D2AF22D185D1E4
:101705007DD17D757701757801757900D1E37C050B
:10171500AD5F1205A6C3ED955F70F5C3E55F940156
:10172500400AC3E55F94FF403202173ED149B1A696
:10173500D185C2AF75EF12D17DDCD50579C3E579C9
:101745009403500280C6D17D0578E5771490009FFB
:1017550093F808C3E57898500280AED17DD17D0518
:1017650077C3E577940A5002809C120EBCB1A6C2DD
:06177500AF75EF12D17DFB
:0319FD00021014C1
:101A00000E0414FFFFFFFF0304090301015AA5019F
:101A1000FFFFFFFFFF03FFFFFF25D0FAFA04FF01DE
:081A2000007AFF01010003FF41
:101A4000235467794B463430412320202020202026
:101A500023424C48454C4923463331302320202033
:101A60002020202020202020202020202020202076
:101C0000C2AFC2D353D9BF7581C043B20343FF8073
:101C1000752438752503B1C975EF0275E24043F1AB
:101C20002053A4DF75D400D2857DFA780379E67C51
:101C300010752200752300901DD67B0675249875BB
:101C400025013085028142208508D8FBD9F9DCF7CF
:101C500081B4308508D8FBD9F9DCF781B4B189E4C7
:101C600093A3C39A6004DDC381B4DBDBB17B600264
:101C7000812B7B08E493FAA3B15CDBF87A30B15C8A
:101C8000752200752300B17BEAFCEBFDC3ED94FEE9
:101C9000400EB17B8A278B28ED30E0048A828B834B
:101CA000B17B7AC270D8C3ED94FE601350CEBD00F4
:101CB00025EC60097520007521FF0200008100A855
:101CC00027A9280809D804D90281D3B17FEA89AAB3
:101CD000F281C50D81A0C3ED94035049EDA2E092BD
:101CE000007AC5C3E5829400E583941C50902000DF
:101CF00010438F02438F0175B7A575B7F1F030001F
:101D00001FA827A9280809438F01538FFDD804D99C
:101D100002A12089AAE275B7A575B7F1F0A3A10DBC
:101D2000538FFC817C7AC1BD030CE493A3FAB140CC
:101D3000DCF8B138817C817EAA22AB23B15CEBFA5E
:101D4000EA6222752608C3E52313F523E52213F57D
:101D50002250066323A0632201D526EAB1C9B1C986
:101D600075260AEAF4200102D285300102C285B14B
:101D7000C9C3134002C201D526EB22B17FEAFB2082
:101D80008502A17F308502A184752608AE24AF2587
:101D9000C3EF13FFEE13FEB1CDB1C9C3EA13308513
:101DA000024480FA30E703632201C3E52313F523DD
:101DB000E52213F52250066323A0632201D526D91C
:101DC000E52265236523F52222AE24AF250E0FDE22
:101DD000FEDFFCD20122424C48656C693437316326
:041DE000F3100601F5
:00000001FF
